:1000000014C02DC02CC02BC02AC029C028C027C0B6
:1000100026C025C040C023C022C021C020C01FC0B0
:100020001EC01DC01CC0280C010611241FBECFED30
:10003000CDBF10E0A0E6B0E0EAE0F3E003C0C89571
:1000400031960D92A836B107D1F710E0A8E6B0E0DE
:1000500001C01D92AA36B107E1F776D055C1D0CFC5
:100060001DBC1CBC81E090E099BD88BDBC9A8FB5D9
:1000700081628FBD8EB589608EBD0895459B03C09A
:100080008FE188BD089581E088BD089588B18864B6
:1000900088B9099A08951F920F920FB60F921124F2
:1000A0002F933F934F935F936F937F938F939F9380
:1000B000AF93BF93EF93FF93E1DFFF91EF91BF9178
:1000C000AF919F918F917F916F915F914F913F91F0
:1000D0002F910F900FBE0F901F901895EF92FF92E7
:1000E0000F931F93CF93DF93ACD0F0906800FF2065
:1000F000F1F08F2DCF2DDD2700E610E0EE2468947F
:10010000E5F8FD2FEC2FE81BF109E00FF11F8081CE
:1001100092D080916800FD2FEC2FE81BF109E00FD1
:10012000F11FE082815080936800882351F762E0DC
:100130008F2D8F5F8DD0F0926800DF91CF911F914E
:100140000F91FF90EF9008958AD0CCD089DF9EDF89
:1001500095DF77D01092680080E0E82FFF27E05A03
:10016000FF4F808168D0809168008F5F8093680026
:10017000883098F362E081E06BD078941092680048
:10018000BED0809369008C3061F08D3021F08A30D0
:1001900079F4A4DFF5CF62E081E05AD010926800D4
:1001A000EFCF4FD062E081E053D010926800E8CFEB
:1001B00080916800883030F091DF62E081E048D0C3
:1001C000109268008091690036D080916800E82F15
:1001D000FF27E05AFF4F9091690090838F5F8093D3
:1001E0006800CECFD19A8B9AD09A8A9A8C9A8D9A9F
:1001F0000895D9989398D8989298992780FDD99A7C
:1002000081FD939A82FDD89A83FD929A949A81E017
:100210008A95F1F7949808951F93182F82958F70FF
:10022000E8DF812FE6DF8DE08A95F1F71F910895D1
:10023000959AF2DF0895FCDF08959598EDDF959A81
:10024000089581E0FADF84EF91E00197F1F70895D6
:100250008150623009F4805C8068EFDF0895EF928E
:10026000FF920F931F93CF93DF93BCDF88E893E156
:100270000197F1F79498959810E0C4EFD1E08C2F96
:100280009D2F0197F1F783E0B4DF1F5F1330B9F7BB
:100290001DE0812F8A95F1F782E0ABDF1A95F1F727
:1002A00086E290E0D92FC82F0F2EF4EFEF2EF1E069
:1002B000FF2EF02D082F192F0D5F1F4FFD2FEC2F54
:1002C000C895802DBADF9F2D8E2D0197F1F72196CD
:1002D0000C171D0799F7DF91CF911F910F91FF9098
:1002E000EF900895599A12B88CE089B988E18AB9DB
:1002F00008955D9BFECF8CB980E090E008955F9BF0
:0A030000FECF8CB199270895FFCFBE
:08030A005465737420302E309D
:00000001FF
